:100000006429B200F839A400A40CA40C240C8407C1
:100010007320B20000055F293208031C03010006AB
:10002000320580065F29A01123080319A0150530A9
:10003000A2002730A900103029200330A900E830A1
:100040002920A90164302920A9010A3029202C087F
:100050003028A8002D08A5002C08A400FA202408A8
:10006000A400A2030319A011230803193A282202AD
:10007000031841282408031DA011A0194128303E6F
:10008000472808000C1E4228990003145F292119F3
:100090004228080083169B0083161C141A089B0A2A
:1000A0005F29A901A800FF30A807031CA907031CAA
:1000B0005F290330A500E5305F205328A501F63EF7
:1000C000A400A509031C6A28FE300000A407031839
:1000D0006528A4070000A50F6428000024187028D4
:1000E00024187228080000308A0032080739820775
:1000F0000134023404340834103420344034803461
:1001000027082F068039B100A71F9128A409A50947
:10011000A609A709A40A0319A50A0319A60A03191F
:10012000A70AAF1F9E28AC09AD09AE09AF09AC0AFA
:100130000319AD0A0319AE0A0319AF0AA801A901F0
:10014000AA01AB01B601B701B801B9012F082E040D
:100150002D042C040319DC282030B0000310A40D5A
:10016000A50DA60DA70DB60DB70DB80DB90D2F082D
:100170003902031DC5282E083802031DC5282D0885
:100180003702031DC5282C083602031CD6282C086C
:10019000B6022D08031C2D0FB7022E08031C2E0FCC
:1001A000B8022F08031C2F0FB9020314A80DA90DC4
:1001B000AA0DAB0DB00BAE28B11FE928A809A909FB
:1001C000AA09AB09A80A0319A90A0319AA0A03195B
:1001D000AB0A3608AC003708AD003808AE00390865
:1001E000AF002808A4002908A5002A08A6002B08AB
:1001F000A7005F29AD01AC011030B000250DAC0D9A
:10020000AD0D2808AC022908031C290FAD02031804
:1002100010292808AC0729080318290FAD07031077
:10022000A40DA50DB00BFE2824085F292030B000D6
:10023000B601B701B801B9010310241C2D292C08FF
:10024000B6072D0803182D0FB7072E0803182E0F19
:10025000B8072F0803182F0FB907B90CB80CB70C43
:10026000B60CA70CA60CA50CA40CB00B1C290800FE
:100270001030B300A501A401B10CB00C031C462939
:100280002808A40729080318290FA507A50CA40C02
:10029000AD0CAC0CB30B3C292C085F29A400A71BA8
:1002A000532124085F29A409A509A609A709A40ABE
:1002B0000319A50A0319A60A0319A70A080083133C
:1002C000831203130000080083160F3099002030BA
:1002D0009800831280309800A001C23083168600F7
:1002E000FD308500073083129F009C2A86156430FC
:1002F0005E20061464305E20861164305E20061095
:1003000064305E2008008615851464305E208611F6
:10031000C921DB21061BC0298519AE294D30422099
:1003200041304220473042204E304220453042206A
:10033000543042203D304220203042200430A10081
:10034000A3013B08AD003A08AC0013202030422046
:100350004220422042200D304220BF294D303A0732
:10036000C2003B080318013EC3004D3042203A084A
:1003700042203B08422042084220430842208A296A
:10038000832985100A305E20080085140A305E201B
:1003900008000930C100C121C5213A30840041085C
:1003A000003E01200310051803140C200130C10287
:1003B0000318CB290800C121C52183100518831417
:1003C00083184014831C4010C121C52183100518D7
:1003D00083148318C014831CC010C121C52183104D
:1003E0000518831483184015831C4011C121C521B1
:1003F0008310051883148318C015831CC011C121F4
:10040000C52183100518831483184016831C4012DD
:10041000C121C5218310051883148318C016831CBD
:10042000C012861514305E2008003B08B1003A085F
:10043000B000A9012D30A8003821C6002D08C70042
:100440004608C4004708C5000730A4000310C50CC7
:10045000C40CA40B262A7F304605C800C9014908F0
:10046000B1004808B000A9010A30A8003821C8002E
:100470002D08C9004808CA004908CB000730A4006D
:100480000310CB0CCA0CA40B402A7F304805C600D1
:10049000C701C708031D502A40304602031C5E2ACC
:1004A0004A08093A4B04031D5B2AC40A0319C50A0A
:1004B000CB01CA015E2ACA0A0319CB0A08005508F3
:1004C0005404031D642A0800A701A6013B08A500E7
:1004D0003A08A400AF01AE010430AD00AC01162112
:1004E0002708D9002608D8002508D7002408D600F8
:1004F0005908A7005808A6005708A5005608A400E8
:10050000AF01AE015508AD005408AC0080202708AB
:10051000D9002608D8002508D7002408D600570897
:10052000BB005608BA0004303B02031C9B2A033070
:10053000BB00FF30BA00080006100330A900E83005
:100540005220CE01CD01CC0101304A20D4004C20F4
:10055000D50003304A20DA004C20DB0086158514D4
:10056000BB01BA0114305E200519B82A762183290F
:10057000861114305E20C9215F228618E42A3B08C8
:10058000AD003A08AC00AE01AF01013EBC00FC304A
:10059000BD002D0803182D0FBD07FF30BE002E082B
:1005A00003182E0FBE07FF30BF002F0803182F0FB0
:1005B000BF073F08A7003E08A6003D08A5003C086D
:1005C0004E21BA002508BB0002304E02031CF42A5B
:1005D0004D08A5004C08A400A9014E08A800FA2067
:1005E000D0002508D100F82A4D08D1004C08D000D1
:1005F0003B085102031C0B2B031D022B3A0850022F
:10060000031C0B2B3A085002D2003B08031C013E8E
:100610005102D300132B50083A02D2005108031C98
:10062000013E3B02D300D308031D1A2B04305202B3
:10063000031C212B3B08CD003A08CC000130CE0032
:100640002C2B0F304E0203182C2B3A08CC073B08FA
:100650000318013ECD07CE0ADB2101305120C01D19
:10066000332B0612352B06160616401E392B861222
:100670003B2B86168616061B892B8519692B15229E
:10068000413042205A304220493042204D304220F1
:100690005530422054304220483042202030422001
:1006A0003D304220203042200430A100A301450803
:1006B000AD004408AC0013202E304220A3014B08AB
:1006C000AD004A08AC001320203042200D304220FB
:1006D000862B41304C07B4004D080318013EB5008D
:1006E0004E083407C20035080318013EC3004130EC
:1006F00042204C0842204D0842204E084220420829
:10070000422043084220CE01CD01CC01061B892B9B
:08071000862BAE2A63008A2B40
:02400E00223F4F
:0A4200000000D300020000000400DB
:00000001FF
